:100000000C9437080C947E080C947E080C943430C1
:100010000C947E080C947E080C947E080C947E0848
:100020000C947E080C947E080C94D2240C940E241C
:100030000C942A280C947E080C947E080C947E085C
:100040000C947E080C947E080C947E080C947E0818
:100050000C947E080C94AC270C947E080C947E08BB
:100060000C947E080C947E080C947E080C947E08F8
:100070000C947E080C947E080C947E080C947E08E8
:100080000C947E080C947E080C947E080C947E08D8
:100090000C947E080C947E080C947E080C947E08C8
:1000A0000C947E080C947E080C947E087B147B14C0
:1000B000B514B51408152415ED16ED16661544167D
:1000C000551655161D224422E6234422E6238C228F
:1000D000AF22E623AA23BD23DB2ADB2AEE2AEE2A5F
:1000E000E42AEE2AEE2AEE2ADB2ADB2AE92AEE2A85
:1000F000EE2AE92A000101010101010101010202C8
:1001000002020202020202030303030303030304C5
:100110000404040404040505050505060606060690
:10012000070707070708080808090909090A0A0A4A
:100130000B0B0B0C0C0C0D0D0D0E0E0E0F0F0F10EC
:100140001011111112121313141415151616171776
:10015000181819191A1A1B1B1C1D1D1E1E1F2020E2
:10016000212222232424252626272829292A2B2C2C
:100170002D2D2E2F30313232333435363738393A4F
:100180003B3C3D3E3F404142434445464748494A47
:100190004C4D4E4F50515354555658595A5B5D5E15
:1001A0005F616264656668696B6C6D6F70727375B0
:1001B00077787A7B7D7E8082838587888A8C8E8F14
:1001C00091939596989A9C9EA0A2A3A5A7A9ABAD42
:1001D000AFB1B3B5B7BABCBEC0C2C4C6C9CBCDCF30
:1001E000D1D4D6D8DBDDDFE2E4E7E9EBEEF0F3F5DE
:1001F000F8FAFDFFFFAA7F55402223252628292A49
:100200002C2D2F3032333536383A3B3D3E40424379
:100210004547494A4C4E5051535557595A5C5E60B8
:1002200062646668696B6D6F71737577797B7D7FCA
:1002300081838587898A8C8E90929496989A9C9EC9
:100240009FA1A3A5A7A8AAACAEAFB1B3B4B6B8B9E5
:10025000BBBCBEBFC1C2C3C5C6C7C9CACBCCCDCE4D
:10026000D0D1D2D2D3D4D5D6D7D7D8D9D9DADADB30
:10027000DBDBDCDCDCDCDCDDDDDDDDDCDCDCDCDCBC
:10028000DBDBDBDADAD9D9D8D7D7D6D5D4D3D2D2FB
:10029000D1D0CECDCCCBCAC9C7C6C5C3C2C1BFBEE3
:1002A000BCBBB9B8B6B4B3B1AFAEACAAA8A7A5A34E
:1002B000A19F9E9C9A98969492908E8C8A8987850D
:1002C00083817F7D7B79777573716F6D6B696866EC
:1002D0006462605E5C5A5957555351504E4C4A49BE
:1002E00047454342403E3D3B3A3836353332302F66
:1002F0002D2C2A29282625232200AF0000000017D4
:1003000000150008001A0014002942000000000A2D
:100310000009000700160004002A61E100E1000561
:1003200000190006001B001D00E10029422C412895
:10033000644C00E300000000000000000000001C0E
:100340000018000C00120013003102000000000B26
:10035000000D000E000F0033003400E100E1001139
:100360000010003600370038002D0028412C422BA9
:10037000002A00E60000000000000000000000313C
:100380000230022F021F021E020100000000003591
:10039000002702260221022002010001000100358F
:1003A0000230002F002302220201002E0033000140
:1003B000000100010000000000000000000000013A
:1003C0000001000100010001003100000000002ECA
:1003D000022D003800250222023400010001002411
:1003E000022E003600370038002D002E00330001A9
:1003F00000010001000000000000000000000022D9
:1004000000210020001F001E00010000000000A9C4
:1004100000AB00AE00AC000100010001000100AA29
:1004200000A800010001000100010001000100011D
:100430000001000100000000000000000000002397
:1004400000240025002600270001000000000050C5
:1004500000510052004F000100010001000100F2B4
:1004600000F100F000F300010001000100010001B3
:100470000001000100000000000000000000003E3C
:10048000003D003C003B003A00010000000000C3BA
:100490005CC95CC55CC75CC25C010001000100C4B2
:1004A0005CCA5CC65CC85C0100010001000100017F
:1004B0000001000100000000000000000000003FFB
:1004C0000040004100420043000100000000000124
:1004D000000100010044004500010001000100018D
:1004E0000001000100010001000100010001000104
:1004F000000100010000000000000000DA12818FFE
:10050000D9F1DB40A4A62EAF00A0C000A1C800AE68
:10051000D580A83FD300408D142000808182838441
:1005200085868788898A8B8C8D8E8F909192939403
:10053000A0A1A2A3A4A5A6A7A8A9AAABACADAEAF43
:10054000B0B1B2B3B4C0C1C2C3C4C5C6C7C8C9CABA
:10055000CBCCCDCECFD0D1D2D3D4002020202020E0
:100560002020005343524C434B20002020202020C9
:100570002020004341504C434B20002020202020CD
:100580002020004E554D4C434B2000556E6465664F
:10059000696E65640A0041646A7573740A00526189
:1005A0006973650A004C6F7765720A00446566617D
:1005B000756C740A004C617965723A20004B79724F
:1005C000696120726576312E300A0A000000000051
:1005D0000000000000000000008080C0E0F07078A3
:1005E000383C1C1E0E0E0E070707070707070707F4
:1005F000070707070707070E0E0E1E1C3C3878700A
:10060000F0E0C0808000000000000000000000005A
:1006100000000000000000000000000000000000DA
:1006200000000000000000000000000000000000CA
:1006300000000000000000000000000000000000BA
:1006400000000000000000000000000000000000AA
:10065000000000C0E0F07C3E1F0F07030180C0E0F7
:10066000F078383C1C1E0E0E070787E77F1FFFFF40
:100670001F7FE78707070E0E1E1C3C3878F0E0C08E
:10068000800103070F1F3E7CF0E0C0000000000067
:10069000000000000000000000000000000000005A
:1006A000000000000000000000000000000000004A
:1006B000000000000000000000000000000000003A
:1006C000000000000000000000000000000000002A
:1006D000F0FCFF1F07010000C0F0FCFEFFF7F3B1C4
:1006E000B03030303030303078FE87010000FFFF0E
:1006F00000000187FE7830303030303030B0B1F358
:10070000F7FFFEFCF0C0000001071FFFFCF0000037
:1007100000000000000000000000000000000000D9
:1007200000000000000000000000000000000000C9
:1007300000000000000000000000000000000000B9
:10074000000000000000000000000000000000FFAA
:10075000FFFF0000000000FEFFFF0101071E78E11F
:1007600081838386868C8C9898B1B7FEF8E0FFFF72
:10077000E0F8FEB7B198988C8C8686838381E17807
:100780001E070101FFFFFE0000000000FFFFFF0049
:10079000000000FFFF0000C0C030300000F0F0009B
:1007A0000000000000F0F00000F0F0C0C030303079
:1007B00030C0C000003030F3F30000000000003013
:1007C0003030303030C0C00000000000000000FFBA
:1007D000FFFF00000000007FFFFF8080E0781E87A1
:1007E00081C1C16161313119198DED7F1F07FFFF93
:1007F000071F7FED8D191931316161C1C181871EDC
:1008000078E08080FFFF7F0000000000FFFFFF0016
:100810000000003F3F03030C0C30300000000033A9
:1008200033333333330F0F00003F3F00000000002D
:10083000000000000030303F3F303000000C0C332F
:1008400033333333333F3F0000000000000000002B
:100850000F3FFFF8E0800000030F3F7FFFEFCF8DD9
:100860000D0C0C0C0C0C0C0C1E7FE1800000FFFF2B
:10087000000080E17F1E0C0C0C0C0C0C0C0D8DCFBD
:10088000EFFF7F3F0F03000080E0F8FF3F0F000005
:100890000000000000000000000000000000000058
:1008A0000000000000000000000000000000000048
:1008B0000000000000000000000000000000000038
:1008C0000000000000000000000000000000000028
:1008D00000000003070F3E7CF8F0E0C08001030732
:1008E0000F1E1C3C38787070E0E0E1E7FEF8FFFF77
:1008F000F8FEE7E1E0E0707078383C1C1E0F07035B
:100900000180C0E0F0F87C3E0F070300000000000B
:1009100000000000000000000000000000000000D7
:1009200000000000000000000000000000000000C7
:1009300000000000000000000000000000000000B7
:1009400000000000000000000000000000000000A7
:10095000000000000000000000010103070F0E1E50
:100960001C3C3878707070E0E0E0E0E0E0E0E0E04F
:10097000E0E0E0E0E0E0E070707078383C1C1E0ED3
:100980000F0703010100000000000000000000004C
:100990000000000000000000000000000000000057
:1009A0000000000000000000000000000000000047
:1009B0000000000000000000000000000000000037
:1009C00000000000000000000000000000AE000475
:1009D0007F3F1F643214643214783C1E1E140A05D3
:1009E00005010902A10185020901A10005091901FA
:1009F00029051500250195057501810295017503ED
:100A000081010501093009311581257F950275089D
:100A1000810609381581257F950175088106050C29
:100A20000A38021581257F950175088106C0C00529
:100A3000010980A10185031A81002A8300160100A3
:100A4000260300950175108100C0050C0901A10164
:100A500085041A01002A9C02160100269C029501B9
:100A600075108100C005010906A101050719E029DB
:100A7000E71500250195087501810295017508812A
:100A8000010507190029FF150026FF0095067508C6
:100A90008100050819012905950575019102950147
:100AA00075039101C009023B00020100A0FA09048C
:100AB0000000010301010009211101000122400091
:100AC0000705810308000A09040100010300000072
:100AD0000921110100012285000705820320000A77
:100AE0001201100100000008EDFE000001000102EB
:100AF00003010403300000001E034B007900720064
:100B00006900610020004B006500790062006F0001
:100B100061007200640000001003730070006C003C
:100B2000690074006B006200000004030904000007
:100B3000000000003E5B4F5B3E003E6B4F6B3E0093
:100B40001C3E7C3E1C00183C7E3C18001C577D5708
:100B50001C001C5E7F5E1C0000183C180000FFE7B4
:100B6000C3E7FF00001824180000FFE7DBE7FF00E1
:100B700030483A060E00262979292600407F0505CF
:100B80000700407F05253F005A3CE73C5A007F3E66
:100B90001C1C0800081C1C3E7F0014227F2214002D
:100BA0005F5F005F5F0006097F017F000066899537
:100BB0006A0060606060600094A2FFA29400080474
:100BC0007E04080010207E20100008082A1C08005F
:100BD000081C2A0808001E10101010000C1E0C1E05
:100BE0000C0030383E383000060E3E0E0600000085
:100BF0000000000000005F00000000070007000088
:100C0000147F147F1400242A7F2A120023130864FF
:100C10006200364956205000000807030000001CFF
:100C2000224100000041221C00002A1C7F1C2A00D7
:100C300008083E0808000080703000000808080816
:100C400008000000606000002010080402003E510F
:100C500049453E0000427F40000072494949460034
:100C60002141494D33001814127F10002745454596
:100C700039003C4A494931004121110907003649F0
:100C800049493600464949291E0000001400000069
:100C90000040340000000008142241001414141411
:100CA00014000041221408000201590906003E41C7
:100CB0005D594E007C1211127C007F494949360073
:100CC0003E41414122007F4141413E007F49494927
:100CD00041007F09090901003E41415173007F082D
:100CE00008087F0000417F4100002040413F010093
:100CF0007F08142241007F40404040007F021C02D8
:100D00007F007F0408107F003E4141413E007F0983
:100D1000090906003E4151215E007F09192946005C
:100D200026494949320003017F0103003F4040400A
:100D30003F001F2040201F003F4038403F00631409
:100D4000081463000304780403006159494D43000B
:100D5000007F414141000204081020000041414150
:100D60007F000402010204004040404040000003B4
:100D7000070800002054547840007F28444438007D
:100D8000384444442800384444287F00385454549C
:100D9000180000087E09020018A4A49C78007F08AF
:100DA0000404780000447D4000002040403D0000E5
:100DB0007F102844000000417F4000007C0478043C
:100DC00078007C0804047800384444443800FC1857
:100DD0002424180018242418FC007C0804040800AB
:100DE00048545454240004043F4424003C40402010
:100DF0007C001C2040201C003C4030403C0044282B
:100E0000102844004C9090907C004464544C440062
:100E1000000836410000000077000000004136085D
:100E200000000201020402003C2623263C000000D0
:100E300000000000404040F0F8F8FF38FFF8F83FAD
:100E4000F8F8FF38FFF8F8F04040400000000000DC
:100E50000080C0C0C0800000C0C08000000080C012
:100E6000C000C0C0000080C0C00000000000C0C0C2
:100E7000C0C0C000C0C000000000000000000000B2
:100E80000000000000000000000000000000000062
:100E90000000000000000000000000000000000052
:100EA00000000000000000000000000000C0F0F89A
:100EB000FC3E1E06010000007F4141417F007F4152
:100EC00041417F000080C0E07E5B4F5BFEC00000C0
:100ED000C000DCD7DEDEDED7DC00C0000000000092
:100EE0000000000000000000000000000000000002
:100EF00000000000494949FFFFFFFFE0DFBFBF00DE
:100F0000BFBFDFE0FFFFFFFF4949490000000000CD
:100F10001F3F6060E0BF1F007F7F071E381E077FF6
:100F20007F007F7F0E1F3B716000000000007F7F0D
:100F30000C0C0C007E7E007F7E0303007F7E03038B
:100F40007E7E03037F7E000F3E703C063C703E0FAA
:100F500000327B49493F7E007F7E0303001E3F69CC
:100F6000696F2600000000000000000000030F1F52
:100F70003F3C7870600000007F4141417F007F412D
:100F800041417F00307B7F7830202030787F3B00EC
:100F900003000F7F0F0F0F7F0F0003000000000002
:100FA0000000000000000000000000000000000041
:100FB00000000000010101070F0F7F0F7F0F0F7E60
:100FC0000F0F7F0F7F0F0F070101010000000000CE
:100FD000000000000001010000000000000000000F
:100FE0000000000000000000000000000000000001
:100FF00000000000000000000000000000000000F1
:1010000000000000000000000000000000000000E0
:1010100000000000000000000000000000000000D0
:1010200000000000000000000000000000000000C0
:1010300000000000000000000000000000000000B0
:1010400000000000000000000000000000000000A0
:101050000000000000000000000000000000000090
:10106000000000000000000000000000000011244B
:101070001FBECFEFDAE0DEBFCDBF04B603FE27C050
:1010800080910C0790910D07A0910E07B0910F076A
:101090008730904BA740B04BD1F410920C071092C0
:1010A0000D0710920E0710920F0714BE84B7877FAA
:1010B00084BF0FB6F894A8958091600088618093F2
:1010C0006000109260000FBEE0E0F8E3099527E0B1
:1010D000A8E8B1E001C01D92AC30B207E1F711E021
:1010E000A0E0B1E0E2ECF5E602C005900D92A83870
:1010F000B107D9F70E944C1A0C94DF320C9400000F
:101100000895BF92CF92DF92EF92FF920F931F93B9
:10111000CF93DF93E82EF62EE901E42FF0E0611182
:1011200006C0EC50FF4F8491B82EE82F71C0262FD7
:1011300030E0EC50FF4FE491FE2FCE2ED12C46E054
:10114000849FC00111240FEF10E0B8010E94973274
:101150004BEA4603C001479F900D11248E0D911D4F
:101160008E0D911D982F990F890FD801A21BB30BDB
:10117000AC9DA001AD9D500DBC9D500D1124B52E10
:10118000F89ED0011124AB2FBB277801EA1AFB0A85
:10119000EC9CD001ED9CB00DFC9CB00D11247801AD
:1011A000E81AF108E29EC001E39E900DF29E900DB8
:1011B0001124892F9927081B190B0C9D90010D9D57
:1011C000300D1C9D300D1124832F6230710591F07C
:1011D00048F461157105E1F061307105B9F48E2FA5
:1011E000EB2F16C06430710569F040F06630710570
:1011F00079F00CC08E2FE52FB32E0AC0E52FBF2E3D
:101200008B2F06C0852FBE2EE32F02C0852FBB2E4D
:10121000E9838883BA82DF91CF911F910F91FF906C
:10122000EF90DF90CF90BF9008959091F20192FFE0
:101230000DC0282F2871283019F4877F846006C0DC
:10124000282F2471243011F48B7F886093FF0DC008
:10125000282F2871283119F4877E846106C0282F31
:101260002471243111F48B7E88612091F30120FFD9
:101270000DC0382F3871383019F4877F816006C06F
:10128000382F3171313011F48E7F886021FF0DC00D
:10129000282F2871283119F4877E816106C0282FF4
:1012A0002171213111F48E7E886194FD877E08952D
:1012B000811106C0662311F089EA09C08AEA07C0D5
:1012C000813039F4662311F08EE401C08BE40C9474
:1012D000642D0895FF920F931F93CF93DF93E091B6
:1012E000EF014E2F440F440F4093EF0120911F0157
:1012F000E22FE295EF70F0E080A190E02F7002C045
:10130000959587952A95E2F78170992750911E014E
:10131000E52FE295EF70F0E020A130E05F7002C0B1
:10132000359527955A95E2F7F901E170FF2720FFDF
:1013300002C0E2E0F0E0E82BF92BE42BE093EF01B0
:10134000F090EE01CF2D0F2C000CDD0BEF70F0E0D4
:10135000E85AFE4F8E010E521E4F9081F801808197
:10136000890F8083843054F0FE01E053FE4F80816A
:101370008F5F808361E08F2D0E945809F801808182
:101380008D3F4CF4C053DE4F88818150888360E0EC
:101390008F2D0E945809F8018081837887FF03C050
:1013A00081508C6F8F5FF8018083DF91CF911F9107
:1013B0000F91FF9008951F93CF93DF93CDB7DEB7C2
:1013C00067970FB6F894DEBF0FBECDBF4B8B5C8B1B
:1013D0006D8B7E8B8F8B86E09E01235F3F4FD90103
:1013E000E82F1D92EA95E9F795E0FE017396D90181
:1013F00001900D929A95E1F7F901DE01179601909F
:101400000D928A95E1F7CE0107960E94F22A81118A
:101410003EC086E0FE013796DE01119601900D92E6
:101420008A95E1F7FF81E8856A857B8561157105FD
:1014300031F0EF3F31F481E0FF3F19F403C081E068
:1014400001C080E080FD23C02091A00630E0C901EA
:101450000196877099274091D10650E0841795072F
:1014600079F1F983EA837D836C8396E0929FD001C2
:10147000939FB00D1124AF55B94FFE0131960190E5
:101480000D929A95E1F78093A0060E94572A16E0E4
:101490008091D1069091A0068917F9F0189FC0019C
:1014A00011248F55994F0E94F22A8823B1F0809120
:1014B000D10690E00196877099278093D106E8CFF6
:1014C0000E94DD2C1092A0061092D106EAE9F6E007
:1014D00086E0DF011D928A95E9F767960FB6F894CA
:1014E000DEBF0FBECDBFDF91CF911F910895209138
:1014F000D7013091D8012817390771F09093D8019E
:101500008093D701E091F501F091F601309721F039
:101510000084F185E02D099408952091D501309142
:10152000D6012817390771F09093D6018093D50121
:10153000E091F501F091F601309721F00680F781F6
:10154000E02D09940895E091F501F091F6013097AE
:1015500021F00190F081E02D099480E008950E942F
:10156000FC27DC01CB01805A9541AF4FBF4F8093E0
:10157000460290934702A0934802B093490280919B
:101580004A0281110BC062E070E089EF92E00E9494
:10159000E420892B19F481E080934A0280914A0269
:1015A0000895EDE6F2E011828281846082830895DD
:1015B00030910D018091680280FF16C0E091EC012E
:1015C00063E0E69FF0011124EC56FE4F539A8BB175
:1015D000877F9BB198602FB7F894AF0163E0369F87
:1015E000400D511D11240BC0E4E9F1E0118210827D
:1015F0001282339681E0E03DF807C1F7DFCFE417B0
:10160000F50789F0319168E09BB9000000C037FF11
:101610008BB9330F000000C000C000C08BB900C000
:101620006A9591F7ECCF2FBF87EC90E00197F1F727
:1016300000C000000895EF92FF920F931F93CF9385
:10164000DF938C01C4E9D1E0E12CF12CF801848115
:10165000FAE0EF16F1041CF4882339F002C081117E
:1016600004C09E0140916B0202C09E0140E0609167
:101670006A02809169020E9481088FEFE81AF80AD5
:10168000239694E1E916F10409F70E94D80AF801BB
:10169000848190E00196817099278483DF91CF91B6
:1016A0001F910F91FF90EF900895EF92FF920F938B
:1016B0001F93CF93DF93EC018C819D810196817004
:1016C00099279D838C8384E9E82E81E0F82E10E031
:1016D00005E5212F26958C819D81820F911D8170BA
:1016E000970140916B0260916A02809F802D1124C6
:1016F0000E9481081F5F83E0E80EF11C143149F756
:10170000DF91CF911F910F91FF90EF900C94D80A29
:10171000EF92FF920F931F93CF93DF937C01FC0115
:101720008481811109C081E084831092920192E04A
:1017300090930C0180930B01C4E9D1E0FE0111826A
:1017400010821282339681E0E03DF807C1F700E095
:1017500010E080919201082E000C990B08171907D0
:1017600094F080910C01082E000C990B80179107C2
:1017700054F09E0140916B0260916A02809169026F
:101780000E94810803C0198218821A820F5F1F4FBE
:10179000239604311105E9F60E94D80A80910B01C5
:1017A00090919201980F9093920120910C01280F33
:1017B00020930C01121614F493313CF08195809320
:1017C0000B01813011F4F7011482DF91CF911F9149
:1017D0000F91FF90EF9008959F92AF92BF92CF929A
:1017E000DF92EF92FF920F931F93CF93DF93EC0161
:1017F0008A8180FF03C0BB24BA9402C0BB24B39487
:101800008C8181110BC081E0B81204C083E1809308
:10181000910102C01092910181E08C8324E9E22EB3
:1018200021E0F22E00E010E034E1932EF701118266
:101830001082128294E0C92ED12CA12C80919101AA
:101840008A0D85312CF0692D0E948932892F02C0C2
:1018500087FD8C5E082E000C990B0817190791F470
:1018600080916B028C9DA0018D9D500D112455958A
:10187000479555954795970160916A028091690255
:101880000E948108AB0CF1E0CF1AD108B9F60F5FC6
:101890001F4F83E0E80EF11C0431110539F60E9458
:1018A000D80A8091910191E0B9120CC0811105C054
:1018B00083E1809391011C820DC08150809391013E
:1018C000BC8208C090E00196B8010E94AB328093C0
:1018D00091018C83DF91CF911F910F91FF90EF9039
:1018E000DF90CF90BF90AF909F900895EF92FF92BE
:1018F0001F93CF93DF93EC0184E9E82E81E0F82E6B
:1019000010E08C81970140916B0260916A02810F17
:101910000E948108145F83E0E80EF11C103F89F7F4
:101920000E94D80A9A818C8190FF02C08F5F01C00B
:1019300081508C83DF91CF911F91FF90EF9008959C
:101940009091680290FF0CC0E4E9F1E0818360832C
:101950004283339691E0E03DF907C1F70C94D80A31
:1019600008950F931F93CF93DF9300D01F92CDB7AD
:10197000DEB78C018091930181110AC09E012F5F17
:101980003F4F4FEF6FEF0E9481088A818093930150
:10199000F8018481813051F028F0823061F4409167
:1019A00093010AC08091930140E007C060919301C8
:1019B00040E080E003C040E080E060E00E94A00CD6
:1019C000F801848190E0019663E070E00E94AB3200
:1019D00084830F900F900F90DF91CF911F910F9103
:1019E0000895CF93DF9300D01F92CDB7DEB79091CB
:1019F000680290FF0AC09E012F5F3F4F0E9481083E
:101A00004B8169818A810E94A00C0F900F900F90EA
:101A1000DF91CF910895CF93DF93EC01E8E6F2E0F8
:101A2000438162818C810E94F10C8C818F5F8C8359
:101A3000DF91CF910895CF93DF93EC01EC81F0E03B
:101A4000E750FE4F4491E8E6F2E0628181810E9416
:101A5000F10C8C818F5F8C83DF91CF910895809101
:101A6000680280FF02C08695089580E00895809105
:101A70006802282F269530E02115310519F4817070
:101A8000826005C02532310524F08170886480931E
:101A900068020895CF92DF92EF92FF926B017C0172
:101AA0000E94370DB701A60188E090E0FF90EF900B
:101AB000DF90CF900C945B325F926F927F928F9207
:101AC0009F92AF92BF92CF92DF92EF92FF920F93CD
:101AD0001F93CF93DF9300D01F92CDB7DEB7182F9F
:101AE000762E042F622E9091680290FF7EC0E92F1F
:101AF000E695AE2FB0E0AD5CBE4F8C9180936D0249
:101B00009E7F923061F49E012F5F3F4F812F0E9494
:101B100081084B8169818A810E94A00C43C0823078
:101B200019F400916B023EC0863019F410916902DD
:101B300039C08930D9F38931A9F5E9518E2F8170E7
:101B4000582EE695F0E0EC50FE4FA590B49084E955
:101B5000C82E81E0D82EE12CF12CBB2494E1892EF3
:101B6000912CAE9CC001AF9C900DBE9C900D112499
:101B7000B4010E949732812F511002C0860F01C01C
:101B8000861B9601402F672D0E9481088FEFE81A6F
:101B9000F80A83E0C80ED11C84E1E816F10409F7C5
:101BA0000E94D80A80916902181308C080916A02C5
:101BB000781204C080916B02081729F080916F029F
:101BC000826080936F021093690270926A020093A0
:101BD0006B02662051F060916802709169028091F9
:101BE0006A0290916B020E944A0D0F900F900F9025
:101BF000DF91CF911F910F91FF90EF90DF90CF90E9
:101C0000BF90AF909F908F907F906F905F9008955E
:101C1000E8E6F2E083E0808311828FEF82838383A2
:101C20001482ADE6B2E012968C9112978360129600
:101C30008C9360817181828193810C944A0D809193
:101C40009001811112C08091D80080618093D800EA
:101C50008AE18A95F1F700C08091D90080FD02C029
:101C600082E001C081E08093900181E09091900139
:101C7000913009F080E00895CF93DF93E72FF0E0F3
:101C800028E0829FE00DF11D1124C3E0EE0FFF1F3D
:101C9000CA95E1F7E60FF11DEE0FFF1FE550FD4F6E
:101CA000C591D491CE01C238D10569F1B0F4C133E8
:101CB000D10509F475C048F4C932D10509F469C0E9
:101CC000CA32D10509F473C079C0C533D10509F40E
:101CD00059C0C933D105B9F071C0C33ED10571F106
:101CE00038F4C03ED105B1F0C23ED10511F166C055
:101CF000C63ED105B9F1C73ED105C9F1C43ED105F3
:101D000009F05CC024C02091F20120FD1AC221FD1F
:101D100018C21CC22091F20120FD0DC22091F301D6
:101D200020FF14C28091F20184FDB7C183EE90E0E0
:101D30000DC22091F20122FF09C2F4CF8091F2017D
:101D400082FDFCC18091F30180FDFBC1EBCF2091AE
:101D5000F30121FFFBC18091F20184FD9EC187EE5A
:101D600090E0F4C12091F20123FFF0C1F4CF809103
:101D7000F20183FDE9C18091F30181FFECCF84EE94
:101D800090E0E4C12091F20125FFE0C189E290E0FA
:101D9000DDC12091F20125FFD9C185E390E0D6C1D4
:101DA0002091F20126FFD2C18AE290E0CFC12091BA
:101DB000F20126FFCBC181E390E0C8C1C11530E537
:101DC000D30708F049C0C11540E4D40708F030C17A
:101DD000C83ED10520F5C03ED10508F0B7C1C83ACC
:101DE000D10570F4C53AD10508F0ADC0C130D105B8
:101DF00009F4ACC108F451C1249708F44EC1A6C13E
:101E0000CF3BD10508F4AAC0C03CD10508F445C1B8
:101E1000CE01880F991FFC01EC58F040FEC0C1159F
:101E200020E2D20760F4C11531E0D30708F08EC17B
:101E3000C03FD10508F431C1CE01906587C1C115FD
:101E400040E3D40708F0ECC0CE019F70FC01EE0F18
:101E5000FF1FEC50FF4FE1C0C11585E5D80708F022
:101E600045C0C11594E5D90708F0FAC0C11522E5AF
:101E7000D20718F5C11531E5D30708F0DDC0CE0152
:101E800074E0969587957A95E1F7282F23703C2F7B
:101E9000337081E090E002C0880F991F3A95E2F715
:101EA0009C68922BEC2FEF70E695E69530E2E39F6D
:101EB000F00111248E2B9F2B49C1AE014370552791
:101EC0002C2F26952695C115D34508F0BAC081E080
:101ED00090E002C0880F991F4A95E2F740E2249FE4
:101EE00090011124822B932B9C6830C1C11599E578
:101EF000D90798F4C11528E5D20708F0B6C0C11576
:101F000036E5D30708F0C9C08C2F0E9415098F71E0
:101F100090E0982F8827906219C1C1154AE5D4072F
:101F200008F4A8C0CE0190568115904208F0B5C0C3
:101F30008D2F8F710E941509FE01FF27F0628F71AE
:101F40009F01382BA8C0C53AD10509F4A9C0C63AEB
:101F5000D10509F0A8C082E890E4F8C0C83AD105DC
:101F600009F4A4C0C93AD10509F4A3C0CA3AD105FD
:101F700009F4A2C0CB3AD10509F4A1C0CC3AD105ED
:101F800009F4A0C0CB3BD10509F49FC0CC3BD105DF
:101F900009F49EC0CD3AD10509F49DC0C03BD105DE
:101FA00009F49CC0CE3AD10509F49BC0CF3AD105C3
:101FB00009F49AC0C13BD10509F499C0C23BD105CF
:101FC00009F498C0C33BD10509F497C0C43BD105BF
:101FD00009F496C0C53BD10509F495C0C63BD105AF
:101FE00009F494C0C73BD10509F493C0C83BD1059F
:101FF00009F492C0C93BD10509F491C0CD3BD1058C
:1020000009F490C0CE3BD10509F48FC0CA3BD1057D
:1020100009F48EC080E094E499C08591949196C0B3
:10202000CE019927D3FF02C0986C90C0906C8EC0EF
:10203000CE019F70906A8AC09C2F8827816F906A1A
:1020400085C081E090E002C0880F991F4A95E2F7B1
:1020500040E2249F90011124822B932B9A6876C032
:102060009C2F8827846F906A71C09C2F8827806F6F
:10207000906A6CC08C2F8F700E941509FE0194E04D
:10208000F695E7959A95E1F7EF70F0E0FE2FEE27D1
:10209000F0699F01282BC90159C080E090E056C02B
:1020A00081E890E453C083E890E450C082EE94E469
:1020B0004DC089EE94E44AC08AEE94E447C085EBB3
:1020C00094E444C086EB94E441C083EB94E43EC0C6
:1020D00084EB94E43BC087EB94E438C08CEC94E44C
:1020E00035C08DEC94E432C083E895E42FC08AE8D3
:1020F00095E42CC082E995E429C084E995E426C0E2
:1021000081E296E423C083E296E420C084E296E470
:102110001DC085E296E41AC086E296E417C087E205
:1021200096E414C08FE694E411C080E794E40EC0F6
:102130008AE296E40BC089E390E008C082EE90E06A
:1021400005C080EE90E002C086EE90E0DF91CF9176
:1021500008950F931F93CF93DF93C62FD42F122F81
:10216000FC0182818823C9F06093D9010E9408286C
:102170009093D4018093D30180E28C0F883008F0D3
:1021800057C0C77081E001C0880FCA95EAF7DF9198
:10219000CF911F910F910C94F32C8091D90168136A
:1021A00030C08091D3019091D4010E94D227883C05
:1021B000910538F500E20D0FCD17B9F080E28C0FD4
:1021C000883040F4C77081E001C0880FCA95EAF7F3
:1021D0000E94E82C083028F581E09D2F977001C0FF
:1021E000880F9A95EAF70E94F32C812F0E94642DA4
:1021F0000830F0F4D77081E001C0880FDA95EAF773
:102200000AC080E28C0F883098F4C77081E001C06A
:10221000880FCA95EAF7DF91CF911F910F910C9427
:10222000E82C812FDF91CF911F910F910C94642D99
:10223000DF91CF911F910F9108956091680266958B
:1022400070E04BE050E080E091E00E94C532892BC5
:1022500019F481E080936E020E9408289093630233
:102260008093620280916F02846080936F02089570
:102270009091680290FF3BC09170811102C0926002
:1022800006C0853210F0986402C0880F982B909396
:10229000680280916F02816080936F02662351F023
:1022A000609168027091690280916A0290916B025C
:1022B0000E944A0D60916802669570E04BE050E024
:1022C00080E091E00E94C532892B19F00E94D10A6A
:1022D00002C00E941D1181E08093650220E04091C0
:1022E0006B0260916A02809169020C945C0D089502
:1022F00061E00C943811809168028695815009F450
:1023000084E261E00C9438118091680286958F5FB9
:10231000853208F081E061E00C9438114F925F92B1
:102320006F927F928F929F92AF92BF92CF92DF92E5
:10233000EF92FF920F931F93CF93DF9368E671E0C4
:102340000BE811E02FE8822E21E0922ED801512CCB
:10235000EE24E394F12C5D017C901C92EB018991B9
:10236000BE01E82FE295EF70F0E021A18F70A70188
:1023700002C0440F551F8A95E2F7CA01242B21A3FE
:1023800022A1442E4094242122A350EA5A95F1F729
:1023900090E7C92E91E0D92E40E050E0E601699027
:1023A0006E01262D22952F7030E0E90128A130E042
:1023B000D62DDF7002C035952795DA95E2F720FD1E
:1023C00007C09701042E01C0220F0A94EAF702C049
:1023D00020E030E03C91232B2C934F5F5F4F48303F
:1023E0005105E1F691A1D42DD923D1A392A1892B36
:1023F00082A3119681E0F5019081971101C080E0E0
:10240000582AF1E0AF38BF0709F0A5CFD091F1010C
:10241000552049F081E080938A010E94082890931A
:1024200089018093880180918A018823A9F0809195
:102430008801909189010E94D227069768F0ED2FBC
:10244000F0E0E850FE4FD8018D918D0181938A16FE
:102450009B06C9F710928A010E941F0E882309F477
:1024600062C0D091F00180916F028823E9F085E08D
:10247000E8E6F2E0ADEDB1E001900D928A95E1F76A
:1024800080916D0290916E02A0916F028093E201A3
:102490009093E301A093E40181E090E00E94C430B6
:1024A000892B11F410926F0280E090E00E94C430FA
:1024B000892B09F0B7C0ED2FF0E0E850FE4F80E027
:1024C00090E0DC01AA51BE4F2C91219301968430FB
:1024D0009105B9F7F090ED010F2D10E000531E4F5C
:1024E000D091EA01F8018081D81BED2E1E1454F41E
:1024F000EA94D8018C918F5F8C9361E08F2D0E94BC
:102500005809F4CF8D2FD7FD80E0D81BDD2309F4C7
:102510009AC0DF5FF80180818150808360E08F2D59
:102520000E945809F3CFE091F1010E2F10E0809145
:10253000E501883009F04CC08091E40180FF25C09E
:102540009091DD018091680290FF0AC081608093C4
:1025500068028091DD0160E086950E94381115C007
:102560008E7F809368020E94D10A80916F02816001
:1025700080936F02FFEF20E742E0F150204040409F
:10258000E1F700C000000E94D80A8091E40181FFB9
:1025900009C020E04091E0016091DF018091DE01FF
:1025A0000E945C0D8091E40182FF09C08091E301EB
:1025B000882319F00E941D1102C00E94D10A809147
:1025C000E40183FF03C081E0809365021092E5017E
:1025D000F801E850FE4F80E090E02191DC01AA5123
:1025E000BE4F2C93019684309105B9F7E091EE012E
:1025F000F0E0E053FE4F80818093EA010E946A0977
:10260000852DDF91CF911F910F91FF90EF90DF907B
:10261000CF90BF90AF909F908F907F906F905F9082
:102620004F90089580918F018F5F80938F01863046
:1026300028F3E091F001F0E0E850FE4F10821182A3
:1026400012821382DBCF10928F01D8CF8F929F928C
:10265000AF92BF92CF92DF92EF92FF920F931F93B0
:10266000CF93DF9300D000D01F92CDB7DEB7FC012F
:10267000D080118183819481892B39F01F3F39F4F7
:1026800091E00FEFD01203C003C091E001C090E0D1
:1026900090FDF0C67F0185E0DE01119601900D925C
:1026A0008A95E1F7F701228189819A81222349F0F5
:1026B0000E942C29082F682F89819A810E94A529C0
:1026C00003C00E947929082FE12FF0E018E0019F54
:1026D000E00DF11D112423E0EE0FFF1F2A95E1F715
:1026E000ED0DF11DEE0FFF1FE550FD4F059114910B
:1026F000033F2CE51207A9F180F4083D8CE518078B
:10270000C9F0093D9CE51907C1F1073DECE51E073D
:10271000B9F526E241EE61EE10C0053FFCE51F076A
:1027200041F118F1063F3CE5130751F527E245EE6C
:1027300066EE03C027E245EE65EEC7010F900F90ED
:102740000F900F900F90DF91CF911F910F91FF90FD
:10275000EF90DF90CF90BF90AF909F908F900C94B0
:10276000A91026E241EE60EEE8CF27E245EE64EEE6
:10277000E4CF26E241EE62EEE0CF28E241E0DCCF9A
:10278000F7018281882309F457C31092D9010D3CC7
:10279000FCE51F0709F4BAC4D0F5023C3CE5130779
:1027A00009F468C6C0F406319CE5190778F40230D4
:1027B000ECE51E0708F0F9C40115FCE51F0709F454
:1027C0008AC301301C4509F059C0B4C306311C4509
:1027D00009F054C01FC60B3C8CE5180778F4053C83
:1027E0009CE5190708F046C6033CECE51E0709F412
:1027F000F6C3043C1C4509F041C008C40B3C2CE561
:10280000120709F45BC40C3C1C45C1F55DC4043DD2
:102810008CE5180709F4A6C4B8F4003DECE51E07E2
:1028200009F486C448F40E3C2CE5120709F470C480
:102830000F3C1C4519F574C4023D8CE5180709F4DA
:1028400087C408F47DC48CC40D3DECE51E0709F473
:10285000A8C448F4053D2CE5120709F48BC40C3DCF
:102860001C4561F49BC40E3D8CE5180709F46BC34D
:10287000C8018A5F9C45099708F497C4F701008155
:102880001181C8010E942C29D82E682FC8010E94EE
:10289000A529B8018D2D0E943C0E8C01982EF701C0
:1028A000A580A2949FE0A922D280D1101092FC06AC
:1028B0008091FA06877079F0DD2069F080E2800F60
:1028C000883048F082E00E94132A8091FA068770CF
:1028D000CC24C3948111C12CB12EB2948FE0B822C4
:1028E0008B2D90E08C30910508F077C2FC01EA5AFC
:1028F000FF4F0C94BF32812F807F1F70882311F00F
:102900001295107FDD20B9F0112309F451C280E245
:10291000800F883010F0911006C08091FD06182BB2
:102920001093FD0605C08091FC06182B1093FC0641
:102930000E94FF283DC2802F0E94FD2C112309F424
:102940004CC2005E1095083010F0911006C08091C6
:10295000FD0618231093FD0605C08091FC06182380
:102960001093FC060E94FF2838C2812F807F1F70C1
:10297000803211F01295107F992021F0F1E09F161E
:10298000E1F02AC0DD2081F08091FE06AA2051F0FE
:1029900001E0A01207C0182B181709F41EC21093EB
:1029A000FE061BC2812B10C0AA2021F021E0A21636
:1029B00009F413C20E94F92827C0DD2041F035E058
:1029C0003A1508F40AC2812F0E94F32C06C284E053
:1029D0008A1508F402C218C0DD2049F0AA2099F334
:1029E000F701858180FFE4C18F708583ECCFAA2039
:1029F00059F0093309F0EEC1FFEF17EE23E0F15073
:102A000010402040E1F7E4C1812F0E94E82CE5C18D
:102A1000812F86958695837019F0813059F0DDC13C
:102A2000DD2019F0C801937002C080E090E00E94A0
:102A30008D0AD9C1DD2019F0C801937002C080E071
:102A400090E00E94770ACFC1DD20F9F0053F51F0F8
:102A5000063F71F0043FA9F48091DB019091DC0105
:102A600081600BC08091DB019091DC01826005C028
:102A70008091DB019091DC0184609093DC01809374
:102A8000DB01802F0E9444271EC0053F51F0063F06
:102A900071F0043FA9F48091DB019091DC018E7FFD
:102AA0000BC08091DB019091DC018D7F05C080918E
:102AB000DB019091DC018B7F9093DC018093DB0143
:102AC000802F0E947D260E9414288DC1812F837043
:102AD00009F069C0D11085C1902F92959695977095
:102AE000990F990F802F8F70882E912CA12CB12CCB
:102AF000092E04C0880C991CAA1CBB1C0A94D2F78E
:102B000004FF12C04FE050E060E070E004C0440FEA
:102B1000551F661F771F9A95D2F7DB01CA01809572
:102B20009095A095B09503C080E090E0DC011695EB
:102B30001695412F4370423019F1C8F40091FF06F9
:102B4000109100072091010730910207413059F0A0
:102B500088299929AA29BB29BC01CD0160237123A9
:102B6000822393230AC0802A912AA22AB32ABC0175
:102B7000CD01682979298A299B290E944D2A31C1D2
:102B800088299929AA29BB290091FF0610910007DD
:102B90002091010730910207BC01CD016027712708
:102BA00082279327EACFDD2019F0812F817001C0A1
:102BB0008695882309F415C1902F92959695977064
:102BC000990F990F802F8F70882E912CA12CB12CEA
:102BD000092E04C0880C991CAA1CBB1C0A94D2F7AD
:102BE00004FF12C04FE050E060E070E004C0440F0A
:102BF000551F661F771F9A95D2F7DB01CA01809592
:102C00009095A095B09503C080E090E0DC0116950A
:102C10001695412F43704230D9F068F500910002BB
:102C2000109101022091020230910302413059F0CB
:102C300088299929AA29BB29BC01CD0160237123C8
:102C4000822393231EC0802A912AA22AB32A13C06A
:102C500088299929AA29BB29009100021091010213
:102C60002091020230910302BC01CD01602771273F
:102C70008227932706C0BC01CD01682979298A29BA
:102C80009B290E94D029ADC01F70DD2039F0812F13
:102C90000E942C2A802F0E94F32CA3C0802F0E9418
:102CA000E82C812F0E94EE299CC0802F32EF9316D2
:102CB00009F440C0391538F090EF991661F0E1EF52
:102CC0009E1699F170C0F3EF9F16D9F124EF92167A
:102CD00009F44EC068C0DD2019F134E03A1508F45B
:102CE0007CC01F7181E090E0A0E0B0E0AC01BD01CC
:102CF00004C0440F551F661F771F1A95D2F78091A5
:102D0000000290910102A0910202B09103028A0197
:102D10009B01082719272A273B27C901B80125C08D
:102D200025E02A1508F459C0DCCFDD2029F0812FD9
:102D30008F712CC0DD20D9F3812F8F710E94EE2975
:102D40004CC0DD2079F01F7181E090E0A0E0B0E0A0
:102D5000BC01CD0104C0660F771F881F991F1A950B
:102D6000D2F703C060E070E0CB010E94D02935C0EB
:102D7000DD2079F01F71812F0E942C2A38E0139FEB
:102D8000C001112483608093FA06812F0E942C2AAF
:102D900024C081E00E94132A81E08A15F0F482E0C9
:102DA0000E94132A1AC0DD2039F0AA2009F4BFCFEF
:102DB000802F0E94772D11C0AA2009F4BDCF89333E
:102DC00049F49FEFE7EEF3E09150E040F040E1F787
:102DD00000C00000802F0E94FD2C88EF8B0D8430F6
:102DE00010F40E94A30ACC2009F444C38091FA068F
:102DF00080FD40C3F70112828595859585950E94D7
:102E00002C2AC7010E9426138091FA068595859584
:102E100085950F900F900F900F900F90DF91CF91AD
:102E20001F910F91FF90EF90DF90CF90BF90AF90E8
:102E30009F908F900C94EE29063CFCE51F0709F447
:102E400005C1F8F406313CE5130709F4F3C250F468
:102E500001159CE5190708F4D5C202301C4508F09D
:102E6000D1C208C3053CFCE51F0708F0E6C0033CDF
:102E70002CE5120708F0FEC2023C1C4509F0C2C254
:102E800075C0063D8CE51807E0F40B3C9CE519077E
:102E900008F0F0C2083CECE51E0709F4E7C008F4AE
:102EA000DEC0093C2CE5120709F4EAC00A3C1C45C7
:102EB00009F0A8C240916B0228E0421B08F440E0F0
:102EC000E5C00C3D8CE5180708F49CC20F3D1C457D
:102ED00008F098C2CFC20E94DD2CEFEFF4E30CE0C3
:102EE000E150F0400040E1F700C0000081E0809335
:102EF000E00080E28093D8001092C9008FE19EE448
:102F00000197F1F700C0000087E090EBDC018093AF
:102F10000C0790930D07A0930E07B0930F079CE04A
:102F200088E10FB6F894A895809360000FBE909347
:102F30006000FFCF80915602982F909590FB80F90A
:102F40008093560297C20F900F900F900F900F90A2
:102F5000DF91CF911F910F91FF90EF90DF90CF9075
:102F6000BF90AF909F908F900C94962880916802AC
:102F700080FF30C08E7F80936802609168027091FC
:102F8000690280916A0290916B020E944A0D0E9430
:102F9000D10A80916F02816080936F029FEFE0E71A
:102FA000F2E09150E040F040E1F700C000000F90E7
:102FB0000F900F900F900F90DF91CF911F910F9175
:102FC000FF90EF90DF90CF90BF90AF909F908F9049
:102FD0000C94D80A8160809368028695CCC0809159
:102FE000FD068272B9F00F900F900F900F900F9026
:102FF000DF91CF911F910F91FF90EF90DF90CF90D5
:10300000BF90AF909F908F900C947B118091FD06A4
:10301000827249F30F900F900F900F900F90DF91F5
:10302000CF911F910F91FF90EF90DF90CF90BF90C5
:10303000AF909F908F900C9484118091690221E051
:1030400040916B0260916A02885F25C0809169029D
:1030500021E040916B0260916A0288501CC060912F
:103060006A0228E0620F08F46FEF06C060916A02FE
:1030700028E0621B08F460E021E040916B0209C087
:1030800040916B0228E0420F08F44FEF21E060917D
:103090006A02809169020F900F900F900F900F902D
:1030A000DF91CF911F910F91FF90EF90DF90CF9024
:1030B000BF90AF909F908F900C945C0D80916C02AC
:1030C000833048F48F5F05C080916C02882319F02B
:1030D000815080936C0260916802709169028091C6
:1030E0006A0290916B020F900F900F900F900F90CB
:1030F000DF91CF911F910F91FF90EF90DF90CF90D4
:10310000BF90AF909F908F900C944A0D81E033C098
:103110000E942F0D8250833008F47CCF82E02BC0B8
:103120000E942F0D8650823008F474CF86E023C0B1
:103130000E942F0D8950853008F46CCF89E01BC0A8
:103140000E942F0D8F50853008F464CF8FE013C09C
:103150000E942F0D8551823008F45CCF85E10BC0B1
:1031600088E109C00E942F0D8951893008F452CF9F
:1031700089E101C083E20F900F900F900F900F90A4
:10318000DF91CF911F910F91FF90EF90DF90CF9043
:10319000BF90AF909F908F900C9478111092080779
:1031A00069C182E08093080765C10E948B28811164
:1031B00002C00E9496280E947A289093F30180937F
:1031C000F20100312CE5120709F4C3C008F041C038
:1031D00008308CE5180709F49AC0F0F40430ECE5E7
:1031E0001E0709F487C068F402302CE5120709F4C1
:1031F00077C003301C4509F0E5C08091F201826080
:1032000076C006308CE5180709F46EC008F07BC064
:103210008091F20188606BC00C30ECE51E0709F468
:1032200085C068F40A302CE5120709F474C008F070
:1032300079C00E94DD2C8091F201806858C00E3068
:103240008CE5180709F476C008F07FC08091F20180
:103250008BC00B3FECE51E0709F44FC018F5033196
:103260002CE5120709F47DC078F401318CE51807CC
:1032700009F473C002311C4509F0A4C00E94DD2C82
:103280008091F2018F7733C00531ECE51E0709F418
:1032900072C008F486C00A3F1C4509F093C08091B3
:1032A000F3013EC00F3F3CE5130709F45FC058F43B
:1032B0000D3F9CE5190709F444C008F43FC0809114
:1032C000F30182602DC00130FDE51F0709F475C0D0
:1032D00008F45DC002301D4509F074C060E06EC0A6
:1032E0008091F201816003C08091F201806180933E
:1032F000F20168C08091F20111C08091F3018260F7
:103300008093F3015FC08091F2018062F0CF8091E1
:10331000F2018064ECCF8091F20188608460E7CF95
:103320008160EECF8091F2018E7FE1CF8091F2013A
:103330008D7FDDCF8091F201877FD9CF8091F3011E
:1033400018C08091F3018D7FDBCF8091F2018F7ED9
:10335000CECF8091F2018F7DCACF8091F2018F7B19
:10336000C6CF8091F201877F8B7FC1CF8091F3011F
:103370008D7F8E7FC5CF8091F20182FB222720F9BD
:1033800091E0922790FB82F990FB83F9B0CF809176
:10339000F301982F909591708E7F892B90FB81F986
:1033A000AFCF0E94DD2C8091F20187FB222720F90C
:1033B00091E0922790FB87F99ACF61E08EE090E050
:1033C0000E9449326091F2011091F30184E090E093
:1033D0000E944932612F81E290E00E9449320F90B1
:1033E0000F900F900F900F90DF91CF911F910F9141
:1033F000FF90EF90DF90CF90BF90AF909F908F9015
:103400000C94DD2CF70100811181C8010E947929FB
:10341000D82E3FCA8091FD068A7A91E009F490E0A7
:103420009093DA01811122C069E282E996E00E945C
:10343000602809C08091DA0181111AC069E282E92D
:1034400096E00E9453280F900F900F900F900F90CE
:10345000DF91CF911F910F91FF90EF90DF90CF9070
:10346000BF90AF909F908F900C94FF2865E3DDCFC5
:1034700065E3E5CF0F900F900F900F900F90DF91C5
:10348000CF911F910F91FF90EF90DF90CF90BF9061
:10349000AF909F908F900895CF93DF93CDB7DEB715
:1034A0002C970FB6F894DEBF0FBECDBF84B7877FD1
:1034B00084BF0FB6F894A8958091600088618093CE
:1034C0006000109260000FBE80E88093610010924F
:1034D000610085B7806885BF85B7806885BF0E9419
:1034E00052240E9471248091E20084608093E20063
:1034F000789480917D028823A1F01091E9001F70DB
:103500009091EC00892F817090FD80E8182B10922B
:10351000E9008091E80083FD0E9439211F7010931B
:10352000E90082E084BD93E095BD9AEF97BD80935A
:103530006E000E941F0E809320018091200188233D
:1035400021F01092EC018AE003C08AE08093EC0144
:1035500080930D010E941F0E62E070E0882329F025
:103560008EE091E00E94E22F04C08EE091E00E9484
:10357000EB2F8091200180912001811102C094E005
:1035800001C090E09093F10184E0891B8093F001E9
:10359000A8E6B1E04CE651E061E070E08D91E82FE3
:1035A000E295EF70F0E021A18F708B0102C0000F57
:1035B000111F8A95E2F7C801902F9095922391A34D
:1035C00092A1892B82A34A175B0741F7A0E7B1E0DC
:1035D00048E751E061E070E08D91E82FE295EF70EF
:1035E000F0E021A18F708B0102C0000F111F8A959E
:1035F000E2F7C801902F9095922391A392A1892B75
:1036000082A34A175B0741F780E0A82E82E0B82E1C
:10361000E8EFF1E01192AE16BF06E1F70E948B28A9
:10362000811102C00E94962880912001811106C05C
:1036300085E380931F0186E680931E0180911F0120
:10364000E82FE295EF70F0E031A1282F2F7081E094
:1036500090E0AC0101C0440F2A95EAF7242F209591
:10366000232321A320911F01E22FE295EF70F0E0C8
:1036700042A12F70BC0102C0660F771F2A95E2F7A6
:103680009B01242B22A320911E01E22FE295EF70D3
:10369000F0E031A12F70AC0101C0440F2A95EAF788
:1036A000242F2095232321A320911E01E22FE295B0
:1036B000EF70F0E032A12F7001C0880F2A95EAF771
:1036C000832B82A320911F01E22FE295EF70F0E09F
:1036D00080A190E02F7002C0959587952A95E2F71A
:1036E000817090911E01E92FE295EF70F0E020A12A
:1036F00030E09F7002C0359527959A95E2F720FD3E
:1037000002C090E001C092E0892B8093EF0190917C
:10371000200181E098279093EE01891B8093ED01B1
:1037200082E08093440280E8809387020E944731C0
:103730006DE070E08EE095E00E94E420892B09F0B6
:1037400043C08091440263E070E081FD3AC08BE0A9
:1037500095E00E94E420892BB9F56DE070E08BEFD5
:1037600094E00E94E420892B79F50E94FC27DC017B
:10377000CB01805A9541AF4FBF4F80934602909343
:103780004702A0934802B0934902EAE8F2E080E0E1
:1037900094E0DF018C011D9201501040E1F7F0939D
:1037A0009106E09390068FEF9FEF909389028093AC
:1037B000880281E080934B0280934A021092450276
:1037C00003C088E095E0C5CF0E948B28811102C01C
:1037D0000E94962882E090E00E9435328093560243
:1037E0000E947A289093F3018093F20183E090E0A5
:1037F0000E943532682F70E080E090E00E944D2AF0
:103800008091F401811138C00E948B28811104C07D
:103810000E9496280E94080E88E090E00E943D32A7
:10382000609368027093690280936A0290936B02BE
:1038300080916F02836080936F026E7F71F40E94AB
:10384000080E88E090E00E943D3260936802709319
:10385000690280936A0290936B020E94370D0E9466
:10386000D10A8091680280FF04C060E086950E94C2
:10387000381181E08093F40188E291E09093F601A1
:103880008093F501CC24C394D12C80917D028530A6
:1038900009F038C080917D02843021F11092F70147
:1038A00020E488E190E00FB6F894A895809360003A
:1038B0000FBE2093600083B7817F846083BF83B78E
:1038C000816083BF7894889583B78E7F83BF0FB65E
:1038D000F894A895809160008861809360001092B0
:1038E00060000FBE80917C02882309F4CECF0E9435
:1038F0008E11E8EFF1E08191811192C3AE16BF06FF
:10390000D1F7C3CF0E948E11982E0E941F0E8823DC
:1039100009F448C0A7E5B2E0E8EFF1E0E12CF12CB2
:103920007E2D61912D912627A9F180E090E030E075
:10393000A901082E02C0559547950A94E2F740FF69
:1039400025C089837A83960102C0220F331F8A958E
:10395000E2F78901862F90E08223932321E0892BCF
:1039600009F420E02B830E9408288160782F9D8332
:103970008C8349815A816B818D810E94DB09F7011B
:10398000E95AFD4F8081082700831CC001968830CA
:10399000910571F63FEFE31AF30A48E0E416F104EB
:1039A00009F0BECF8FEF8E838F8318860E94082880
:1039B0008160782F9A8789874E815F8168858A85A3
:1039C0000E94DB0980914B02882309F4C4C18AE874
:1039D00092E090939106809390060E941F0E882398
:1039E00009F48DC08BE195E00E94D6208DEB95E027
:1039F0000E94D62085EB95E00E94D62040910002DF
:103A0000509101026091020270910302CB01AA273A
:103A1000BB270097A105B10521F0AC01BD0180E1F4
:103A200001C080E0052F162F272F33270115110520
:103A30002105310519F0885FB901A8018A019B01B0
:103A4000A4E03695279517950795AA95D1F7011506
:103A500011052105310519F08C5FB901A8018A0112
:103A60009B01F2E03695279517950795FA95D1F7C2
:103A7000011511052105310519F08E5FB901A80165
:103A80007695679557954795452B462B472B09F01B
:103A90008F5F813059F038F0823059F0833061F413
:103AA00086E995E00BC08CEA95E008C085EA95E0D0
:103AB00005C08EE995E002C08BE895E00E94D62013
:103AC0000E94A30A182F80FD03C08BE795E002C077
:103AD00083E895E00E94D62011FD03C08BE695E0B7
:103AE00002C083E795E00E94D62012FD03C08BE55B
:103AF00095E002C083E695E00E94D62029C020917F
:103B0000880230918902AAE8B2E080E090E0AC013E
:103B10004F5F5F4FFA01E453FA4FE4916C91E6175F
:103B200071F0EC9366E0969587956A95E1F7B6019A
:103B300002C0660F771F8A95E2F7262B372B119666
:103B4000CA014115544019F7309389022093880225
:103B500020918802309189022115310509F4DBC0DA
:103B6000809145028111D7C0282E312C7601082E74
:103B700002C0EE0CFF1C0A94E2F7A7014223532374
:103B8000452B11F48F5FF0CF90914402910106E034
:103B9000220F331F0A95E1F790FD13C08295880F1D
:103BA000880F807480932301220F232F221F330B51
:103BB000319520932601815C809324011092270186
:103BC00012C0B6E036952795BA95E1F7220F220F7D
:103BD000220F2093230110922601295F20932401B4
:103BE00087E08093270124E630E047E050E061E27F
:103BF00071E088E70E94D431892B09F08CC0809154
:103C0000440280FD23C0C101A6E0880F991FAA9538
:103C1000E1F7AC0146575D4F04E610E020E430E0E8
:103C200060E488E70E94FB31892B09F074C00E9490
:103C3000AF0AE094F0948091880290918902E82282
:103C4000F922F0928902E092880265C080E4E4E003
:103C5000F2E0DF011D928A95E9F7F6E0220C331CB1
:103C6000FA95E1F7E0E8F1E0FC87EB8748E751E0FF
:103C7000AB85BC858D91BC87AB87FA019191AF0173
:103C80009101290F311D890106571D4F280190E030
:103C90008C5F9D4FFC0107E09F01281B390B7C2C9A
:103CA00001C0770C2A95EAF7B201812CDB011D9146
:103CB000BD011721202F28192770622E022E000C1B
:103CC000330BB12F01C0BB0F6A94EAF76B2E31950D
:103CD000219531092770332701C016952A95EAF7F7
:103CE000612A1081612A6082839418E08112DECFFC
:103CF000015031960F3F81F628E831E06B857C85D5
:103D00002617370709F0B4CF04E610E020E430E0CE
:103D100044E052E085CF80914A028823E1F0409050
:103D200046025090470260904802709049020E94FB
:103D3000FC27DC01CB0184199509A609B709B7FD59
:103D40000AC062E070E08CEC99E00E94E420892BCC
:103D500011F410924A0291100E94AF0A809153020E
:103D6000909154020E94D227AC019091520291117D
:103D700003C02CE231E002C022E330E042175307D7
:103D800008F478C080914E0210914F0281110BC04F
:103D900011115CC120915002211158C12091510292
:103DA000211154C167C09F3F19F09F5F9093520249
:103DB000181624F40E94242780934E0280914E020C
:103DC00087FF05C00E942427819580934E0211161B
:103DD00024F40E94242780934F0280914F0287FF92
:103DE00005C00E942427819580934F0230914E0296
:103DF0003323E1F020914F022223C1F075EB37030A
:103E0000C0011124992319F090934E0203C081E060
:103E100080934E0205EB2003C0011124992319F071
:103E200090934F0203C081E080934F028091500233
:103E3000181624F40E9402278093500280915002A9
:103E400087FF05C00E9402278195809350028091D0
:103E50005102181624F40E94022780935102809187
:103E6000510287FF05C00E9402278195809351026D
:103E70000E9414280E94A30A90915502891721F0EC
:103E80000E94A30A8093550280916E02882309F450
:103E9000FCCC80916D02E0916802E695E81BE0930E
:103EA0006402823059F4F0E0E452F64FE4910E2FB0
:103EB00010E0EBE1EE2EEDE0FE2E59C0863059F415
:103EC000F0E0E752F64FE4910E2F10E07BE0E72E92
:103ED0007DE0F72E4CC0893061F4E695F0E0EA52BF
:103EE000F64FE4910E2F10E066E7E62E6CE0F62E1A
:103EF0003EC08F3061F4E695F0E0ED52F64FE4916C
:103F00000E2F10E05CEEE52E5BE0F52E30C0853123
:103F100059F4F0E0E053F64FE4910E2F10E048E83A
:103F2000E42E4BE0F42E23C08831A1F0833249F413
:103F3000EEECF9E00591149131EBE32E3CE0F32E29
:103F400016C0843271F404EF11E02BE1E22E2BE075
:103F5000F22E0DC008EE13E095E5E92E9BE0F92E58
:103F600006C000ED17E080E8E82E88E0F82E80918A
:103F70006502882389F0109265020E940828980142
:103F800020953095820F931F909363028093620275
:103F90001092670210926602809162029091630211
:103FA0000E94D2278017910708F46FCC809161029C
:103FB0008823B1F01092610280915F0290916002BB
:103FC0000E94D2278033954758F00E94082890938A
:103FD000600280935F0280916F02886080936F021D
:103FE0008090660290906702E0916202F091630215
:103FF0000E0F1F1F109363020093620282E692E08D
:10400000F70109958091660290916702892B09F06A
:104010003CCC892809F439CC81E08093610235CC0D
:1040200080E189BD82E189BD09B400FEFDCF8091A8
:10403000D8008F7D8093D8008091E00082608093CB
:10404000E0008091E00081FDFCCF1FCC9F3F09F094
:10405000ACCEBDCECF93DF93C0919006D0919106A8
:104060008A30B1F420918702CE018A589240622FA3
:1040700070E00E949732281B822F66E00E947D32FA
:10408000C82FC15008F48FC080E20E942A20F9CFC7
:104090008D30E9F4CA58D24020918702622F70E037
:1040A000CE010E949732281B822F9E01280F311DBE
:1040B0002115344018F080E0C0E0D0E0C80FD11DD9
:1040C000C657DD4FD0939106C09390066CC096E022
:1040D000FE01AAE8B6E001900D929A95E1F7813EC3
:1040E00030F086E0FE0111928A95E9F70BC0F6E008
:1040F0008F9FB0011124625D744F46E050E0CE0105
:104100000E942C32C0919006D091910646E050E07A
:10411000BE018AE896E00E94D232892B49F19E01C5
:104120002A583240A90186E0569547958A95E1F7CD
:1041300081E090E0BC0102C0660F771F4A95E2F76C
:104140004091880250918902462B572B2A5F3F4F9E
:1041500066E0369527956A95E1F702C0880F991FAA
:104160002A95E2F7842B952B9093890280938802FD
:104170009E012458324040918702642F70E0C901AB
:104180000E949732481B463010F4240F311D211530
:1041900084E0380710F020E030E026573D4F3093A0
:1041A000910620939006DF91CF910895CF93DF93EE
:1041B000EC01FE018491882321F00E942A2021969F
:1041C000F8CFDF91CF910895EF92FF920F931F9355
:1041D000CF93DF93EC017B0164E670E088E70E94F7
:1041E0004D318C01EC0EFD1ECE15DF0561F017FD83
:1041F0000AC0FE01849164E670E00E94A4318C0143
:104200002196892B89F30E942832C801DF91CF9132
:104210001F910F91FF90EF900895EF92FF920F93EF
:104220001F93CF93DF937C018B010E94912E81110C
:1042300019C0E70101151105A1F08091E80085FD85
:104240000AC08091E8008E778093E8000E94912E4A
:10425000882381F307C089918093F10001501109EF
:10426000E9CF80E0DF91CF911F910F91FF90EF9008
:1042700008951F93CF93DF93CDB7DEB7AA970FB6FC
:10428000F894DEBF0FBECDBFEFE7F2E08091F10002
:10429000819322E0E738F207C9F7809180028330EA
:1042A00009F460C030F4813071F0823009F49AC0B2
:1042B000B1C08A3009F486C08B3009F46BC08930F4
:1042C00009F0A8C020C080917F02813A09F0A2C005
:1042D0008091E800877F8093E8008091830290912D
:1042E0008402892B21F468E083E792E003C060E058
:1042F00080E090E070E00E94182F8091E8008B77BA
:104300008093E80087C080917F02813209F082C0EB
:104310008091830290918402029708F07BC0809183
:10432000E800877F8093E8008091E80082FD05C067
:1043300080917D028111F8CF6DC02091F3008091B2
:10434000F20090E0922B029729F48091F1008B7F8C
:10435000813021F48091F100809372028091E80015
:104360008B7754C080917F02813A09F053C08091CD
:10437000830290918402892B09F04CC08091E8005F
:10438000877F8093E8008091E80080FFFCCF8091D8
:10439000320137C080917F028132E1F58091830242
:1043A00090918402892BB1F58091E800877F8093FA
:1043B000E8000E94C42E80918102809332010E9405
:1043C000DD2C28C080917F02813221F58091E800A8
:1043D000877F8093E8000E94C42E809182028093A0
:1043E000710218C080917F02813AA1F48091E800A7
:1043F000877F8093E8008091E80080FFFCCF809168
:1044000071028093F1008091E8008E778093E8003C
:104410000E94C42E8091E80083FFD8C180917F0262
:1044200090918002492F50E04A30510508F0CEC1EA
:10443000FA01EE59FF4F0C94BF32803821F08238D8
:1044400009F0C4C108C080917B0290917C0299233D
:1044500089F082600FC0809183028F70873008F0EE
:10446000B5C18093E9008091EB0085FB882780F936
:104470001092E9009091E800977F9093E800809374
:10448000F1001092F10071C1282F2D7F09F09EC11B
:10449000882319F0823061F099C1809181028130C6
:1044A00009F094C1933009F080E080937C022EC023
:1044B0008091810281112AC0809183028F702FEF39
:1044C000280F263008F082C18093E9002091EB008C
:1044D00020FF1CC0933021F48091EB00806214C057
:1044E0009091EB0090619093EB0021E030E0A90106
:1044F00002C0440F551F8A95E2F74093EA001092DC
:10450000EA008091EB0088608093EB001092E90054
:104510008091E800877F2CC1811158C110918102E0
:104520001F778091E3008078812B8093E300809156
:10453000E800877F8093E8000E94C42E8091E80005
:1045400080FFFCCF8091E30080688093E30011112D
:1045500002C082E001C083E080937D0237C18058B1
:10456000823008F033C180918102909182028C3DAB
:1045700053E0950779F583E08A838AE289834FB710
:10458000F894DE01139620E03EE051E2E32FF0E0E4
:1045900050935700E49120FF03C0E295EF703F5F16
:1045A000EF708E2F90E0EA3010F0C79601C0C096F1
:1045B0008D939D932F5F243149F74FBF8091E80081
:1045C000877F8093E8006AE270E0CE0101960E9446
:1045D000182FBAC04091830250918402292F3327AB
:1045E00023303105B1F068F42130310509F4FDC004
:1045F0002230310509F0EAC08BE390E0E5EAFAE009
:1046000050C02132310581F12232310509F439C01F
:10461000DDC0992781309105B9F070F082309105A5
:10462000D9F0039709F0D2C0E2EFFAE0E4918E2FBF
:1046300090E0E2EFFAE032C0EAE2FBE0E4918E2F94
:1046400090E0EAE2FBE02AC0E8E1FBE0E4918E2F93
:1046500090E0E8E1FBE022C0E8EFFAE0E4918E2F81
:1046600090E0E8EFFAE01AC04115510509F4C2C024
:104670004130510509F0AAC089E090E0E0EDFAE090
:1046800010C04115510509F4BAC04130510509F077
:104690009DC085E890E0E0EEF9E003C0009709F4E2
:1046A00095C02091E800277F2093E80020918502A3
:1046B000309186028217930708F49C0140E021158F
:1046C000310589F180917D02882309F43DC0853050
:1046D000D9F18091E80083FD37C08091E80082FD28
:1046E0002FC08091E80080FFEACF4091F3008091D5
:1046F000F20090E0942B2115310559F08830910596
:1047000040F444914093F1003196215031090196D3
:10471000F2CF41E0089709F040E08091E8008E7701
:104720008093E800CCCF4111CDCF0AC080917D02AB
:10473000882351F0853041F08091E80083FD04C06A
:104740008091E80082FFF2CF8091E8008B77809320
:10475000E8003CC08038D1F58091E800877F8093E5
:10476000E80080917E028093F1008091E8008E77CE
:104770008093E8000E94C42E29C0811127C0809137
:104780008102909182029927029704F58091E800B6
:10479000877F8093E8001091810210937E020E942F
:1047A000C42E111106C08091E30087FD02C081E094
:1047B00001C084E080937D0242E061EC81E00E94D0
:1047C000E32E42E261EC82E00E94E32E8091E80059
:1047D00083FF1AC08091E800877F8093E800809172
:1047E000EB0080628093EB000FC082E190E0E0EE8E
:1047F000FAE057CF89E090E0E7EBFAE052CF80E4AF
:1048000090E0E5E6FAE04DCFAA960FB6F894DEBF49
:104810000FBECDBFDF91CF911F9108951F920F92D0
:104820000FB60F9211242F933F934F935F936F9383
:104830007F938F939F93AF93BF93CF93DF93EF9328
:10484000FF93C091E900CF708091EC00D82FD17018
:1048500080FDD0E81092E9008091F000877F80937E
:10486000F00078940E9439211092E9008091F000C4
:1048700088608093F000CD2BCF70C093E900FF914A
:10488000EF91DF91CF91BF91AF919F918F917F91E8
:104890006F915F914F913F912F910F900FBE0F90AD
:1048A0001F901895E8EDF0E080818E7F8083109254
:1048B000E2001092DA001092E100A0EEB0E08C91DC
:1048C00081608C9380818F77808319BCA7EDB0E0E5
:1048D0008C918E7F8C9380818F7E8083109270026A
:1048E0000895CF92DF92EF92FF920F931F93CF9391
:1048F000DF93C8EDD0E088818F7E8883E7EDF0E01C
:1049000080818160808384E082BF81E08093700237
:1049100088818E7F888302EE10E0F8011082109269
:10492000DA0081EEC82ED12CF601108288818F77B3
:10493000888388818068888388818F7D888319BC7B
:1049400010927D0210927E0210927C0210927B02E5
:1049500090EEE92EF12CF70180818B7F8083888196
:104960008160888342E060E080E00E94E32EF601EF
:1049700080818E7F8083F801808181608083808147
:1049800088608083F70180818E7F80838881806149
:104990008883DF91CF911F910F91FF90EF90DF906F
:1049A000CF9008951F920F920FB60F9211242F935C
:1049B0003F934F935F936F937F938F939F93AF93A7
:1049C000BF93EF93FF938091E10082FF09C0809134
:1049D000E20082FF05C08091E1008B7F8093E100BF
:1049E0008091DA0080FF2AC08091D80080FF26C025
:1049F0008091DA008E7F8093DA008091D90080FF69
:104A000018C080E189BD82E189BD09B400FEFDCFF7
:104A100081E080937D028091700281110FC00E941D
:104A200052240E9471248091E20084608093E2000D
:104A300005C019BC10927D02109270028091E100B5
:104A400080FF17C08091E20080FF13C08091E200D8
:104A50008E7F8093E2008091E20080618093E2008B
:104A60008091D80080628093D80019BC85E0809343
:104A70007D028091E10084FF32C08091E20084FFDA
:104A80002EC080E189BD82E189BD09B400FEFDCF61
:104A90008091D8008F7D8093D8008091E1008F7E37
:104AA0008093E1008091E2008F7E8093E20080910C
:104AB000E20081608093E20080917E02882311F001
:104AC00084E007C08091E30087FD02C081E001C05F
:104AD00083E080937D020E94DD2C0E94A30A8091D6
:104AE000E10083FF27C08091E20083FF23C0809113
:104AF000E100877F8093E10082E080937D02109245
:104B00007E028091E1008E7F8093E1008091E2003F
:104B10008E7F8093E2008091E20080618093E200CA
:104B200042E060E080E00E94E32E8091F000886027
:104B30008093F000FF91EF91BF91AF919F918F9182
:104B40007F916F915F914F913F912F910F900FBE89
:104B50000F901F901895809172020895CF93DF9364
:104B600000D01F92CDB7DEB720917D02243031F501
:104B700023E02983805891099B838A8382E0809374
:104B8000E9008FEF9091E800815095FD06C095ED0A
:104B90009A95F1F700008111F5CF8091E80085FF2B
:104BA0000DC040E050E063E070E0CE0101960E944D
:104BB0000D218091E8008E778093E8000F900F9090
:104BC0000F90DF91CF9108950F931F93CF93DF93B1
:104BD00000D01F92CDB7DEB78C010E94762F8230B5
:104BE00011F0843021F584E089831B830A8382E0FD
:104BF0008093E9008FEF9091E800815095FD06C009
:104C000095ED9A95F1F700008111F5CF8091E800BC
:104C100085FF0DC040E050E063E070E0CE010196FA
:104C20000E940D218091E8008E778093E8000F901C
:104C30000F900F90DF91CF911F910F910895CF9317
:104C4000DF93EC010E94762F823011F08430F9F46A
:104C500082E08093E9008FEF9091E800815095FD0C
:104C600006C095ED9A95F1F700008111F5CF80917E
:104C7000E80085FF0CC040E050E066E070E0CE0147
:104C80000E940D218091E8008E778093E800DF91EB
:104C9000CF910895CF93DF93EC010E94762F82305D
:104CA00011F0843039F581E08093E9008FEF909125
:104CB000E800815095FD06C095ED9A95F1F700004A
:104CC0008111F5CF8091E80085FF14C040E050E0ED
:104CD00068E070E0CE010E940D218091E8008E779F
:104CE0008093E80088E0FE01A3E7B2E001900D9216
:104CF0008A95E1F7DF91CF910895803F39F4809153
:104D00004F0287FF6CC010924F0269C0813F29F4A7
:104D100080914F021816BCF362C090914E02823F00
:104D200029F497FF5CC010924E0259C0833F19F4DA
:104D30001916CCF354C0893F41F4809150021816E3
:104D40000CF04DC0109250024AC08A3F29F4809165
:104D5000500287FF44C0F6CF8B3F39F48091510257
:104D600087FF3DC0109251023AC08C3F29F48091D8
:104D700051021816BCF333C0843F21F480914D02D8
:104D80008E7F17C0853F21F480914D028D7F11C029
:104D9000863F21F480914D028B7F0BC0873F21F429
:104DA00080914D02877F05C0883F31F480914D028C
:104DB0008F7E80934D0213C08D3F21F480910707B1
:104DC0008E7F0BC08E3F21F4809107078D7F05C039
:104DD0008F3F29F4809107078B7F8093070780918D
:104DE0004E0281110EC080914F0281110AC0809144
:104DF0005002811106C080915102811102C01092AF
:104E0000520208958091070780FD16C081FD16C0EB
:104E100082FD18C080915202882391F0883290F46C
:104E200028E0829FC001112468E270E00E94AB324A
:104E3000862F672B29F007C082E0089584E008954B
:104E400081E0089588E008958091070780FD14C0EF
:104E500081FD14C082FD16C080915202882381F02A
:104E6000843180F422E3829FC001112464E170E068
:104E70000E94AB32862F08958CE0089589E1089551
:104E800085E0089582E30895803F21F40E9424275D
:104E9000819504C0813F29F40E94242780934F020A
:104EA0000895823F21F40E942427819504C0833F06
:104EB00029F40E94242780934E020895893F19F413
:104EC0000E94022705C08A3F31F40E940227819583
:104ED0008093500208958B3F21F40E940227819510
:104EE00004C08C3F29F40E94022780935102089548
:104EF000843F21F480914D02816017C0853F21F4E9
:104F000080914D02826011C0863F21F480914D0254
:104F100084600BC0873F21F480914D02886005C0FA
:104F2000883F31F480914D02806180934D02089555
:104F30008D3F21F48091070781600BC08E3F21F4E3
:104F400080910707826005C08F3F29F48091070791
:104F5000846080930707089578941F920F920FB68C
:104F60000F9211248F939F93AF93BF938091030768
:104F700090910407A0910507B09106070196A11D25
:104F8000B11D8093030790930407A0930507B09386
:104F90000607BF91AF919F918F910F900FBE0F9019
:104FA0001F901895CF92DF92EF92FF920F931F936D
:104FB0002FB7F894409103075091040760910507BB
:104FC000709106072FBF6A017B01EE24FF248C013C
:104FD00020E030E0C016D106E206F30610F441509E
:104FE00051099A01281B390BC9011F910F91FF909C
:104FF000EF90DF90CF9008952FB7F894609103075A
:105000007091040780910507909106072FBF0895BE
:105010002FB7F8948091030790910407A09105079A
:10502000B09106072FBF0895E091F501F091F601C8
:10503000309749F082E080934C020480F581E02DA6
:105040008CE492E009950E94082890935402809382
:10505000530208951F920F920FB60F9211248F934F
:105060009F93AF93BF938091F701811113C08091FB
:10507000030790910407A0910507B0910607419698
:10508000A11DB11D8093030790930407A09305070A
:10509000B0930607BF91AF919F918F910F900FBE74
:1050A0000F901F9018959C012A5F3F4FFC01428191
:1050B000461301C01282019682179307B9F708952B
:1050C0009C01FC0132969FEF80E04191461789F0E8
:1050D0009F3F19F4411101C0982F8F5F8630A9F7C7
:1050E0009F3F39F0F901E90FF11D97FDFA956283B1
:1050F00008950895CF9384E090E00E943532C82F40
:1051000081E290E00E9435322C2F30E0A901582B2B
:10511000CA01CF91089580E090E00E94433221E0DF
:105120008C3E9E4F09F020E0822F08956CEE7EEFBA
:1051300080E090E00E94673260E082E090E00E94B0
:10514000493260E083E090E00E9449321092FF060D
:1051500010920007109201071092020760E084E0AD
:1051600090E00E94493260E081E290E00E94493282
:1051700060E085E090E00E94493260E086E090E0E7
:105180000E9449326FEF87E090E00E94493240E090
:1051900050E0BA0188E090E00E945B3260E08DE070
:1051A00090E00E94493240E050E0BA0188E190E08E
:1051B0000E945B3260E087E190E00E94493240E06B
:1051C00050E0BA018CE190E00E945B3260E080E246
:1051D00090E00E94493240E050E0BA018FE090E058
:1051E0000E945B3240E050E0BA0183E190E00C9411
:1051F0005B328091FE0681111092FE060895909117
:10520000FD068091FC06892B2091FB06982F922B9E
:10521000909392068091FE06882389F0892B8093D3
:105220009206E4E9F6E097E080E0915029F02191C0
:105230002223D9F38F5FF9CF81110E94F928E091E1
:10524000F501F091F601309731F00280F381E02D05
:1052500082E996E009940895BF92CF92DF92EF928F
:10526000FF920F931F93CF93DF938C01C0900002A6
:10527000D0900102E0900202F09003028091FF06BC
:1052800090910007A0910107B0910207C82AD92A7E
:10529000EA2AFB2ACFE1D0E0D701C6010C2E04C0D8
:1052A000B695A795979587950A94D2F780FD04C087
:1052B000219790F7B12C07C0BC2EB8018C2F0E940B
:1052C0003C0E0197A9F38B2DDF91CF911F910F9188
:1052D000FF90EF90DF90CF90BF900895CF93DF9332
:1052E000EC010E942C29BE010E943C0EDF91CF915F
:1052F000089528E0929F800D1124682F6695669589
:105300006695982F977085E0689FB001112440E062
:1053100050E080E0FB01E40FF51FEE52F94F2081D1
:1053200030E0092E02C0369527950A94E2F72170E5
:105330003327042E01C0220F0A94EAF7822B4F5F15
:105340005F4F4530510531F7089528E0929F800D59
:105350001124E82FE695E695E695877051E001C0A7
:10536000550F8A95EAF785E0E89FF0011124EE5287
:10537000F94F20E030E070E04081CB01022E02C006
:10538000969587950A94E2F7817081958427852305
:10539000842781932F5F3F4F2530310569F70895AA
:1053A0000F931F938B019C0106701127222733272F
:1053B000DC01CB01063011052105310511F48860AF
:1053C00001C0877F8093000290930102A0930202A4
:1053D000B09303021F910F910C94C22C0F931F9353
:1053E00041E050E060E070E004C0440F551F661FCC
:1053F000771F8A95D2F7409550956095709580916A
:10540000000290910102A0910202B09103028A0170
:105410009B01082319232A233B23C901B8011F91AB
:105420000F910C94D0292091FA06809582238093C5
:10543000FA06982F977079F430E0482F082E000C68
:10544000550B2417350739F08595859585950E946C
:10545000EE291092FA0608950F931F9341E050E051
:1054600060E070E004C0440F551F661F771F8A95E7
:10547000D2F78091000290910102A0910202B091B6
:1054800003028A019B01082B192B2A2B3B2BC901F4
:10549000B8011F910F910C94D0296093FF0670936F
:1054A000000780930107909302070C94C22C80910F
:1054B000D1069091A006891719F08F5F8770FBCFF6
:1054C0000895CF9380919F0682958F7009F05FC0F9
:1054D00080919C06882309F45AC08091D106B0912E
:1054E000A00670919A06A0919B0640919D0650914E
:1054F0009E0691E07F3F09F090E0692FC6E08B1790
:1055000009F445C04115510521F0AF3F21F020E0DD
:1055100003C021E001C0262F90E020FD35C0C89FC8
:10552000F001C99FF00D1124EF55F94F21812A1385
:105530002BC02081271328C02281211125C023815F
:1055400034812417350710F421503109241B350B01
:10555000283C3105C8F420919F062F7020612093CC
:105560009F0626E0289FF001299FF00D1124EA559F
:10557000F94F80818F70806180838AE996E00E9474
:105580002613CF910C94572A01968770B8CFCF91EC
:1055900008950E946E29292F2F70E92FE295EF7050
:1055A0004E2F50E0FA013297EE30F105B8F4E4598D
:1055B000FF4F0C94BF32803F99F018F4883E70F48E
:1055C0000FC0843F59F40CC0883E50F0813F31F445
:1055D00007C0822F869586958695089580E0089568
:1055E00081E00895AF92BF92CF92DF92EF92FF9247
:1055F0000F931F93CF93DF93CDB7DEB761970FB6AD
:10560000F894DEBF0FBECDBF8C0185E0F801DE014E
:105610001D9601900D928A95E1F7D8013C91119663
:105620002C9111971296EC9050919A0660919B06DE
:1056300080919D0690919E06009731F06F3F31F466
:1056400041E05F3F19F403C041E001C040E0B42FE6
:10565000B170BB2E40FD43C1F801C380D480A0903F
:105660009C06AA2009F4E2C040919F06C816D906FC
:1056700028F0D601A81BB90BCD0104C080959095E8
:105680008C0D9D1DFF24F394883C910548F0F12C6E
:10569000407F09F090C08AE996E00E94261317C166
:1056A000842F807F09F052C0621312C0531310C0C0
:1056B000FE2CE1100DC04F70406140939F068AE9B7
:1056C00096E00E94261380919F06F801858348C1C9
:1056D000CD2831F02F3F31F481E03F3F19F403C072
:1056E00081E001C080E080FD03C081E08E2502C022
:1056F00080E090E0F82FF170FF2E80FF1CC08091B9
:10570000D1064091A00656E0841709F406C190E046
:10571000589FF001599FF00D1124EF55F94F618109
:10572000261306C06081361303C06281E61203C0EF
:1057300001968770E9CFFE2CEE2009F411C180910B
:105740009F06816080939F06F12C0AC1621308C0F6
:10575000531306C0E11004C080919F06F80199C060
:105760003D872E878D859E850E94C92A882369F1F1
:10577000EE2059F120919F06822F82958F7090E044
:10578000029774F080919A0690919B0698878F8378
:105790001986DB86CA862C87CE0107960E942613BF
:1057A00086E0F801AAE9B6E001900D928A95E1F74A
:1057B0000E94612A0DC0621771F03D872E878D858A
:1057C0009E850E94C92A81111AC0C8010E94261311
:1057D000FF24F394C5C05313F0CFE110EECF8091B6
:1057E0009F06F8018583C8010E94261386E0EAE936
:1057F000F6E0DF011D928A95E9F7FA2CB1C0EE20A0
:1058000021F320919F06822F82958F7090E002975E
:105810003CF280919A0690919B069A8389831B8221
:10582000DD82CC822E83CE010196B8CFC816D90670
:1058300038F0C81AD90AB8ECCB16D10450F007C01A
:10584000809590958C0D9D1D883C910510F0F12C54
:105850003EC0FE2CEE2009F4B8CF621327C05313CC
:1058600025C020919F0620FD18C0822F82958F7041
:10587000482F50E04115510581F0F80125834F3044
:10588000510541F08F5F982F9295907F822F8F70F6
:10589000892B8583C8010E94261386E0F801AAE9B6
:1058A000B6E001900D928A95E1F75AC03D872E87A8
:1058B0008D859E850E94C92A811172CF80919F0695
:1058C000816080939F06C8010E94261349C0EAE9BF
:1058D000F6E086E0DF011D928A95E9F741C0EE20EF
:1058E00009F473CF3D872E878D859E850E94C92A36
:1058F000F82E882309F469CF86E0F801AAE9B6E01A
:1059000001900D928A95E1F780919A0690919B06FD
:105910000E946E290E94612A23C03D872E878D85B3
:105920009E850E946E29292F22952F70223028F4FF
:105930009F7039F0811105C00BC0243028F49F708E
:1059400049F4805E883020F0C8010E942613BF2CE5
:10595000FB2C06C0D80115969C91907F91F7F8CF4B
:105960008F2D61960FB6F894DEBF0FBECDBFDF91CD
:10597000CF911F910F91FF90EF90DF90CF90BF904C
:10598000AF9008951092FC061092FB060E94FF282B
:10599000ECE4F2E086E0DF011D928A95E9F71092CF
:1059A0005202109207070E94142880E090E00E94A3
:1059B0008D0A80E090E00C94770A1092FD0686E054
:1059C000E4E9F6E0DF011D928A95E9F70C94C22C18
:1059D000882341F080959091FD0689238093FD06F0
:1059E0000C94FF280895882339F09091FD06892BA7
:1059F0008093FD060C94FF280895882309F463C062
:105A0000823869F40E94A30A81FF5DC069E382E9DC
:105A100096E00E9460280E94FF2869E30EC0833848
:105A200091F40E94A30A80FF4EC063E582E996E0EC
:105A30000E9460280E94FF2863E582E996E00E94A8
:105A400053280C94FF28843869F40E94A30A82FF2B
:105A50003AC067E482E996E00E9460280E94FF282D
:105A600067E4EBCF9CEF980F913A10F4682FE5CFE5
:105A700090E2980F983088F4877021E030E0A90117
:105A800002C0440F551F8A95E2F7CA018095909194
:105A9000FD0689238093FD06D4CF9BE5980F9330B4
:105AA00020F480E090E00C948D0A98E5980F9731EF
:105AB00020F480E090E00C94770A803F20F00E9470
:105AC0007D260C9414280895CF93C82F0E94772D1B
:105AD000C93349F42FEF87EE93E021508040904086
:105AE000E1F700C000008C2FCF910C94FD2C88238F
:105AF00009F416C18238B1F40E94A30A81FD10C1D5
:105B000069E382E996E00E9460280E94FF282FEF57
:105B100041EE54E0215040405040E1F700C0000009
:105B200069E317C08338D9F40E94A30A80FDF8C046
:105B300063E582E996E00E9460280E94FF288FEFCB
:105B400091EE24E0815090402040E1F700C0000039
:105B500063E582E996E00E9453280C94FF2884387C
:105B6000B1F40E94A30A82FDDBC067E482E996E0FB
:105B70000E9460280E94FF284FEF51EE84E04150C0
:105B800050408040E1F700C0000067E4E2CF9CEFA6
:105B9000980F913A30F4682F82E996E00E946028CD
:105BA000DCCF90E2980F983080F4877021E030E0ED
:105BB000A90102C0440F551F8A95E2F7CA019091CE
:105BC000FD06892B8093FD06C8CF9BE5980F933087
:105BD00070F4853A29F0863A31F083E890E005C008
:105BE00081E890E002C082E890E00C948D0A98E58C
:105BF000980F973108F08EC0883A09F445C0893A69
:105C000009F445C08A3A09F445C08B3A09F445C005
:105C10008C3A09F445C08B3B09F445C08C3B09F430
:105C200045C08D3A09F445C0803B09F445C08E3A21
:105C300009F445C08F3A09F445C0813B09F445C0D9
:105C4000823B09F445C0833B09F445C0843B09F419
:105C500045C0853B09F445C0863B09F445C0873BF8
:105C600009F445C0883B09F445C0893B09F445C0A7
:105C70008D3B09F445C08E3B09F445C08A3B09F4CD
:105C800045C080E090E044C082EE90E041C089EEE3
:105C900090E03EC08AEE90E03BC085EB90E038C0DB
:105CA00086EB90E035C083EB90E032C084EB90E06F
:105CB0002FC087EB90E02CC08CEC90E029C08DECDD
:105CC00090E026C083E891E023C08AE891E020C0FC
:105CD00082E991E01DC084E991E01AC081E292E07E
:105CE00017C083E292E014C084E292E011C085E222
:105CF00092E00EC086E292E00BC087E292E008C01C
:105D00008FE690E005C080E790E002C08AE292E072
:105D10000C94770A803F20F00E9444270C941428AA
:105D200008952091E4003091E50095E64091EC0063
:105D3000842F817040FF23C08091E80080FD1DC04A
:105D400080917D02882399F0853099F08091EB0055
:105D500085FD11C04091E4005091E50024173507FE
:105D600029F3915011F09A01E1CF84E0089582E087
:105D7000089583E0089581E0089580E008954091BA
:105D8000E80042FFDDCF089580917F0287FF11C0B8
:105D90008091E80082FD05C080917D028111F8CFDD
:105DA00011C08091E8008B770BC080917D02882321
:105DB00049F08091E80080FFF8CF8091E8008E776D
:105DC0008093E8000895982F973068F59093E90044
:105DD000981739F07091EC002091ED005091F0008F
:105DE00003C0242F762F50E021FD02C09F5FECCF2F
:105DF0003091EB003E7F3093EB003091ED003D7F22
:105E00003093ED003091EB0031603093EB007093F4
:105E1000EC002093ED005093F0002091EE0027FD60
:105E2000E5CF80E008958F708093E90081E00895C8
:105E300020918502309186022617370748F06115B8
:105E4000710539F42091E8002E772093E80001C015
:105E5000B901FC0120E06115710579F180917D02A5
:105E60008823F1F18530F1F18091E80083FD3CC099
:105E70008091E80082FD2EC08091E80080FFEBCF8A
:105E80002091F3008091F20090E0922B6115710552
:105E900051F08830910538F421912093F100615040
:105EA00071090196F3CF21E0089709F020E0809175
:105EB000E8008E778093E800CECF2111CFCF0AC0C3
:105EC00080917D02882361F0853061F08091E80047
:105ED00083FD0AC08091E80082FFF2CF80E0089540
:105EE00082E0089583E0089581E008958091080795
:105EF000811107C080917D02843011F081E0089506
:105F000082E008958EE14A9B02C08150E1F74A9BEE
:105F1000FECF08955A9880E28A95F1F75A9A08952B
:105F2000FC012AE02A95F1F790E020E080E031E0E2
:105F3000261779F040E14A95F1F7880F4A9B02C095
:105F40008160932700C0000040E14A95F1F72F5F80
:105F5000EFCF20E12A95F1F729B100C0000030E130
:105F60003A95F1F722FB222720F992272081920F00
:105F700090830895EF92FF920F931F93CF93DF9337
:105F80001F92CDB7DEB719828C017C01E60EF11CA1
:105F90000E151F0559F00E94822F68E0CE01019670
:105FA0000E94902FF80181938F01F2CF81E09981B7
:105FB000911180E00F90DF91CF911F910F91FF9091
:105FC000EF90089590930B0780930A076093090759
:105FD000529A5A9A089590930B0780930A076093F8
:105FE000090752985A9AEA9AE9E6F0E080818F7C94
:105FF00080830895615091E001C0990F6A95EAF796
:1060000020E031E0992361F0492F482319F05A9A92
:10601000232701C05A9840E24A95F1F79695F2CFAE
:10602000222311F05A9A01C05A9880E28A95F1F71A
:106030005A980895FF920F931F93CF93DF93EC012B
:106040008C01060F111DC017D10741F0F9900E9475
:106050008A2F68E08F2D0E94FA2FF5CFDF91CF9124
:106060001F910F91FF9008951F920F920FB60F92FC
:1060700011240F931F932F933F934F935F936F932D
:106080007F938F939F93AF93BF93EF93FF93CF93A0
:10609000DF931F92CDB7DEB719820E94822F67E08F
:1060A000CE0101960E94902F382F36953695369561
:1060B000932F96959570232F2570920F292F23707B
:1060C000969596958770920F891348C089818111A2
:1060D00045C080910907831708F440C080E18A9584
:1060E000F1F75A9A529AA2E0AA95F1F700C00091EE
:1060F0000A0710910B07B8E03B9F000D111D1124FA
:106100005A98F8016581662321F0868197810E9463
:106110001A300E948A2FF0E1FA95F1F75A985298B6
:106120005A9A80E18A95F1F7D80112966C911297EC
:10613000662369F013968D919C9114970E94BA2F53
:10614000D801ED91FC91811105C082E004C0D80115
:10615000ED91FC9188E080830E94822F0F90DF9167
:10616000CF91FF91EF91BF91AF919F918F917F91CF
:106170006F915F914F913F912F911F910F910F90D0
:106180000FBE0F901F9018950F931F93CF93DF931F
:106190002091090730E0281739070CF471C09C01E1
:1061A00093E0220F331F9A95E1F7C0910A07D0912F
:1061B0000B07C20FD31FF894529A5A9845E04A959C
:1061C000F1F70000982F969595708570890F982F9C
:1061D000937086958695890F8901082B0E948A2FD6
:1061E00084E08A95F1F700C067E0802F0E94FA2FC3
:1061F00040E14A95F1F752985A9A4A9902C000C074
:10620000FCCF87E090E04A9B0EC0019751F4529A70
:106210005A9AE881F98181E08083789481E090E066
:1062200031C000C0F0CF6D81662381F08E819F81E7
:106230000E94BA2F81110AC0529A5A9AE881F981B4
:1062400082E08083789482E090E01CC00E94822FDC
:1062500080E28A95F1F75A98529A40E14A95F1F70F
:106260006A81662321F08B819C810E941A300E94F2
:106270008A2FE881F9811082789480E090E002C052
:1062800084E090E0DF91CF911F910F9108951092DB
:10629000B9008CE08093B8000895EF92FF920F93BD
:1062A0001F93CF93DF93182FEB011092BC0084EA69
:1062B0008093BC000E9408287C018091BC0087FD6F
:1062C0000EC0CF3F8FEFD807C1F30E9408288E1968
:1062D0009F098C179D0788F38EEF9FEF2EC080914A
:1062E000B900887F883041F08091B900887F803183
:1062F00019F08FEF9FEF21C01093BB0084E88093CB
:10630000BC000E9408288C018091BC0087FD0CC055
:10631000CF3F8FEFD807C1F30E940828801B910B55
:106320008C179D0788F3D8CF8091B900887F88317A
:1063300011F08034F1F680E090E0DF91CF911F9171
:106340000F91FF90EF9008950F931F93CF93DF93DA
:10635000EB018093BB0084E88093BC000E94082876
:106360008C018091BC0087FD0EC0CF3F8FEFD80716
:10637000C1F30E940828801B910B8C179D0788F39E
:106380008EEF9FEF0CC02091B900287F81E090E054
:10639000283211F480E090E0919581959109DF9188
:1063A000CF911F910F910895CF92DF92EF92FF92BC
:1063B0000F931F93CF93DF936B018A017901B9018A
:1063C0000E944D31E6010C0D1D1DC017D10761F46F
:1063D00024E92093BC00DF91CF911F910F91FF9092
:1063E000EF90DF90CF90089597FDF2CFB70189919C
:1063F0000E94A431EACFCF92DF92EF92FF920F93E7
:106400001F93CF93DF93C62F6A017901B8010E94D1
:106410004D3197FD11C0B8018C2F0E94A431E601C7
:10642000EC0CFD1CCE15DF0539F097FD05C0B80159
:1064300089910E94A431F6CF24E92093BC00DF911A
:10644000CF911F910F91FF90EF90DF90CF90089523
:1064500084E98093BC000895FB01DC0102C0059033
:106460000D9241505040D8F70895F999FECF92BD52
:1064700081BDF89A992780B50895A6E1B0E044E07F
:1064800050E00C946F32A8E1B0E042E050E00C9490
:106490006F32262FF999FECF92BD81BDF89A0197F0
:1064A00000B4021639F01FBA20BD0FB6F894FA9A5C
:1064B000F99A0FBE08950396272F0E944A320E9430
:1064C0004932252F0E944A32242F0C944A320196D9
:1064D000272F0E944A320C944932DC01CB01FC0187
:1064E000F999FECF06C0F2BDE1BDF89A319600B42D
:1064F0000D9241505040B8F70895991B79E004C0BF
:10650000991F961708F0961B881F7A95C9F78095F2
:10651000089587FB082E062687FD819567FD619506
:106520000E947D320EF4919507FC81950895AA1B77
:10653000BB1B51E107C0AA1FBB1FA617B70710F06E
:10654000A61BB70B881F991F5A95A9F780959095A0
:10655000BC01CD01089597FB072E16F4009407D0D7
:1065600077FD09D00E94973207FC05D03EF4909544
:1065700081959F4F0895709561957F4F0895EE0F17
:10658000FF1F0590F491E02D0994FC01415050400B
:1065900030F001900616D1F73197CF010895882782
:1065A00099270895FB01DC0104C08D9101908019A9
:1065B00021F441505040C8F7881B990B0895F89476
:0265C000FFCF0B
:1065C20001191A1B1C1D1E1F202122010214EB019E
:1065D20000EB0105E601E50108DD0100000035667A
:1065E200010021007F220007AB254A261F26AE2587
:1065F200E425010001020202020606060909090950
:1066020009090F0F0F0F0F0F151515181919191961
:10661200191919191919232400FF0100010000FF9B
:10662200FF0000010001FF0034C697940000000043
:1066320036323331F7F6F5F40008101820283038D6
:08664200383028201810080070
:00000001FF
